:0200000480007A
:100000006F008004732F2034930F80006308FF0378
:10001000930F90006304FF03930FB0006300FF038E
:10002000130F000063040F0067000F00732F2034CC
:1000300063540F006F00400093E19153171F0000BD
:1000400023223FFC6FF09FFF93000000130100008C
:10005000930100001302000093020000130300004C
:100060009303000013040000930400001305000034
:10007000930500001306000093060000130700001C
:100080009307000013080000930800001309000004
:1000900093090000130A0000930A0000130B0000EC
:1000A000930B0000130C0000930C0000130D0000D4
:1000B000930D0000130E0000930E0000130F0000BC
:1000C000930F0000732540F16310050097020000B4
:1000D000938202017390523073500018970200000F
:1000E00093824202739052309B021000939252030B
:1000F0009382F2FF7390023B9302F0017390023AF5
:100100007350403097020000938242017390523046
:10011000735020307350303093010000970200007C
:10012000938282EE73905230130510001315F5017F
:10013000635C05000F00F00F930110009308D005D9
:10014000130500007300000093020000638A0200A0
:1001500073905210B7B200009B82921073902230BD
:100160007350003097020000938242017390123462
:10017000732540F1730020309306F0061725000028
:10018000031545E8972500008395E5E71300000077
:100190001300000013000000130000001300000013
:1001A0001300000013000000130000001300000003
:1001B00013000000130000001300000013000000F3
:1001C000972200002392A2E497220000239FB2E22C
:1001D0000F10000097270000938707E3678307004D
:1001E000130000009303C01B93012000639A76065E
:1001F000130740061307F7FFE31E07FE97220000D0
:100200002398A2E0972200002395B2E00F1000008F
:100210001300000013000000130000001300000092
:100220001300000013000000130000001300000082
:100230001300000013000000130000001300000072
:10024000972700009387C7DC67830700130000002F
:100250009303903093013000639476006310300272
:100260000F00F00F638001009391110093E11100E2
:100270009308D00513850100730000000F00F00FF4
:10028000930110009308D0051305000073000000CF
:10029000731000C00000000000000000000000001B
:0802A000000000000000000056
:1010000000000000000000000000000000000000E0
:1010100000000000000000000000000000000000D0
:1010200000000000000000000000000000000000C0
:1010300000000000000000000000000000000000B0
:081040000000000000000000A8
:102000009386D6149386E60DE70703009386B622DF
:10201000E7070300000000000000000000000000CF
:040000058000000077
:00000001FF
